:100000000A284F2C582C612CFE00030EF0000A0821
:10001000F100682B0E2D1529BC01B401AC01033091
:10002000B300BB00C3003D1435142D144825A40AA9
:1000300008006E257F30D8000530A7004825A03085
:10004000A5000F30D52821210319260A031D080019
:10005000A030A5000F30A6004825FB24003A031964
:10006000080068257F30D900DC000730A700D030B9
:10007000A5000730D52821210319260A031D0800F1
:10008000D030A5000730A6004825FB24003A03190C
:10009000080068257F30D901DC00BD10B514352873
:1000A00021210319260A031D0800D030A5000730BE
:1000B000A6004825FB24003A0319080062257F307A
:1000C000D4000530362821210319260A031D080013
:1000D000D030A5000730A6004825FB24003A0319BC
:1000E0000800BD30D701D6006225A701A70AD22497
:1000F0000530A500A601A40AAB01AA010800212130
:100100000319260A031D08000530A500A601D22404
:100110002B08031908002A08031908000530AA0152
:10012000AB01A301A2005730A1003030BF28292124
:100130000319210A0319220A0319230A0319AF28F4
:100140000130A5020030031CA603A602250A0319EC
:10015000260A031D08000530A500A601D22CBC010B
:10016000FF30B400AC0048250230C300BB00B30030
:100170000430A7001F30A301A201A1004030A0005D
:10018000172829210319210A0319220A0319230A0E
:10019000031D08004825FB24003A031908006225C6
:1001A0000630A700B830A5000B30A6001728212183
:1001B0000319260A031D0800B830A5000B30A6005D
:1001C0004825FB24003A0319080068250730D12888
:1001D00021210319260A031D0800B830A5000B30A1
:1001E000A6004825FB24003A031908006E250630B6
:1001F000A700B830A5000B30A600A40AAA01AB01E5
:10020000080021210319260A031D0800B830A500A3
:100210000B30A60048252B08031908002A080319EB
:100220000800AA01AB01A4010800240884000C30D6
:1002300004020318080005308A001E3004078200FB
:1002400008000130A5020030031CA603A602250AFF
:1002500008000130D000D101D201D301A002510821
:10026000031C510FA1025208031C520FA202530893
:10027000031C530FA302200A0800CF00063E84008F
:1002800083130008CD00CE008E29C401C40A4F0894
:10029000D122C401C40A4F0820234F08023E56222F
:1002A0004F08013E84000014CE019C294F08A92369
:1002B000CE01CE0A9C294F08A9234F08033E56229F
:1002C000023070294F0896244708C4004F082023A5
:1002D00060294608C4004F08D1224F087424053015
:1002E000CE009C294F08013E8400801C69294F08DC
:1002F00096244708C4004F0820236029642203186D
:100300009C2905308A002A30040782004D08003AF3
:1003100003197E29083A03197E299C294F08073EB4
:1003200084000008013A03198629033A0319542965
:10033000013A031945299C294F08073E8400800192
:100340004E084D0603193E2A4E08CD003E2A4708A6
:10035000C4004F0820230230302A4708C4004F0849
:100360004A244F08033E5622AB294708C4004F08D1
:100370004A24AB295E228014492A64220318492AA0
:1003800005308A003430040782004608C4004F0854
:10039000D1220530302A4708C6294708C4004F0833
:1003A000D1224F08023E5622C9295E228010492AD6
:1003B00064220318492A05308A003E30040782006F
:1003C0004F08033E84000008FF3ECA00FF300318B8
:1003D0000030CB004F0884004B08803ACC008030BE
:1003E0004C02031DF52900084A028312031CFD2953
:1003F0004F0884008313800A492A49080319082AF0
:100400004F08043E84004908831380000330302ADB
:100410000430302A4F08023E84000008013ECA0022
:10042000003003180130CB004F0884004B08803A9D
:10043000803C031D1D2A4A0800028312031C242A43
:100440004F0884008313382A480803192F2A4F08BD
:10045000043E84004808831380000630302A0730A9
:10046000CE00492A69220319082A4F08043E840055
:100470008003492A692203192F2A352A4D0884004E
:10048000093004020318492A05308A005130040754
:1004900082004E084D0603194F2A4E08CD004F0822
:1004A000063E84004D088313800008008400000885
:1004B000CA004F0884004A08800008000830CE00B7
:1004C0004F08013E84000800270884000A30040217
:1004D00008004F08043E840080080800F300F20082
:1004E0000310F20D0310F20D0310720D313E840063
:1004F00073088000C8222C3E84008001C8222D3E53
:1005000084000010C822323E84008001C8222D3EA3
:1005100084008014B52AC8222E3E84008001D701B1
:10052000D501C8222F3E8400FF308000D600D400C1
:10053000C32AC8222E3E84008001DF01DD01C822CB
:100540002F3E8400FF308000DE00DC00C32AC8227A
:100550002E3E84008001DB01D901C8222F3E840099
:10056000FF308000DA00D800C32AC822313E840060
:1005700000088400033004020318C32A05308A00EF
:100580008F3004078200C822303E840080010800BA
:100590007308F2000310F20D0310F20D0310720D38
:1005A0000800C500C4080319F12AFA2A4508023ECA
:1005B00084005608F2005708E5238000080045082B
:1005C000023E84005E08F2005F08E5238000080018
:1005D0004508023E84005A08F2005B08E5238000CB
:1005E0000800450819230318080005308A008030E8
:1005F00004078200440B08000F2B4508023E8400CC
:100600005508800008004508023E84005D0880000F
:1006100008004508023E840059088000080045088B
:1006200019230318080005308A008330040782006C
:100630000800053E8400000884000330040208001E
:10064000C500C4080319402B492B4508033E84000C
:100650005608F2005708E523800008004508033ECD
:1006600084005E08F2005F08E5238000080045086A
:10067000033E84005A08F2005B08E523800008006E
:10068000450819230318080005308A007A3004074A
:100690008200440B08005E2B4508033E840054088A
:1006A000800008004508033E84005C0880000800C4
:1006B0004508033E840058088000080045081923B7
:1006C0000318080005308A007D3004078200080006
:1006D0000B198B1EA22B83122D1C7C2BF90379087E
:1006E000FF3A031D762BFF300511F9002C08790223
:1006F00003187D2B05157D2B0511351C8D2BFA0359
:100700007A08FF3A031D872BFF308510FA00340862
:100710007A0203188E2B85148E2B85103D1C9E2B80
:10072000A8032808FF3A031D982BFF300510A800E6
:100730003C08280203189F2B05149F2B0510B0308E
:100740000B11810071088A00700E8300FE0E7E0E70
:100750000900F400B52B7408023E8400800174087F
:10076000033E8400FF308000BE2B74081923031859
:10077000BE2B05308A008630040782007408023ED2
:10078000DF230008F3007208730274080318CD2BEE
:10079000023EDF2372088000740884000008F20023
:1007A0007408033E84000008F30072087302031803
:1007B00008007408033EDF237208800008008400EC
:1007C0000008F200740884000800F6007B08F300BB
:1007D00005300310F30CFF3E031DE92B7B08F400EA
:1007E0000310F40C0310F40C0310F40C7B08F50058
:1007F0000310F50C0310F50C7508740673067B06E0
:10080000F8000130F8057808F30007300310F30D05
:10081000FF3E0310031D072C7B0C7304FB007608BE
:100820007B027B08031CE72B72027B08031CE72B6F
:10083000F7000800E72400306E2201306E220230FB
:100840006E227425B524851A332CFE30E00563082A
:10085000803A600461046204031D402CA901A90AC6
:10086000AA01AA0A402C6014600A0319610A03193C
:10087000620A7F3003196306031D402CAB01AB0AEB
:100880000310E00DE10DE20DE30D29080319232CFF
:100890000B20232CC500C408031D08006A2C450842
:1008A000033E84005608F2005708E5238000080044
:1008B0004508033E84005E08F2005F08E5238000DF
:1008C00008004508033E84005A08F2005B08E5234F
:1008D00080000800450819230318080000308A002A
:1008E0000130040782000800F300832C73088400A1
:1008F000730884008008031D8C2C73088400FF306B
:1009000080008C2C762C7308192303188C2C05304E
:100910008A00893004078200730884000008F2000E
:100920007308033E8400720880000800F300A22CC4
:10093000730884008008031DAB2C730884008001B9
:10094000AB2C982C730819230318AB2C05308A00A4
:100950008C3004078200730884000008F2007308DA
:10096000023E840072088000080083160F178F165D
:100970000F168F110F1401108110011181158112B2
:100980008312AC0803190511B40803198510BC08BB
:1009900003190510F901FA01A8010B118B168B1729
:1009A0000B1708000A30C601C701C800C9002C3067
:1009B0003D21DF2434303D21DF243C303D296430AB
:1009C000C601C60AC701C70AC800C9000800073027
:1009D000990015089F0183169F01811396018312C8
:1009E00090118316851605118510051083120511C7
:1009F0008510051008003208083A031DB208031DCF
:100A000000343A08083A031DBA08031D00344208AE
:100A1000083A031DC2080319013400342030F901DB
:100A2000FA018313840044305A25FF30E000E100CE
:100A3000E200E300E130FB0083011A2C0C281928A6
:100A400023283B28502863287F289728C128D728A7
:100A5000E82801295B296229622969295629622926
:100A60006929722962296929AD29A729B529AD29E2
:100A7000492A492ABA29BA29BA29B529CD29C52925
:100A8000CD29CB29492AD529492AD529CB29D529A8
:100A9000DF242C303D21DF2434303D21DF243C3065
:100AA0003D29492A492AE029322AD8290A2A3A2AFC
:100AB000BD29492A64008001840A04060319003410
:100AC00004065B2D0230C300BB000130B3000800F8
:100AD0000130C300BB000230B30008000130C30086
:100AE0000230BB00B30008000430A501A601A70036
:100AF000A4010800252B2E2B372B4C2B522B582BC7
:100B0000D62ADF2AE82AFD2A032B092BAB2BAB2B95
:100B1000AB2B762C822C822C982CA12CA12C8B2AEE
:040B2000992AA72A3D
:02400E00E4F0DC
:00000001FF
